:1000000041C07AC158C057C056C055C054C053C033
:1000100052C051C050C04FC04EC04DC04CC04BC06C
:100020004AC049C048C009021200010100801909F4
:10003000040000000000000012011001FF00000891
:10004000C016DC0500010102000116035500530033
:1000500042006500780061006D0070006C00650072
:10006000200363006F006400650061006E0064009F
:100070006C006900660065002E0063006F006D0073
:100080000403090411241FBECFEDCDBF10E0A0E68C
:10009000B0E0E4E3F6E002C005900D92A237B107AC
:1000A000D9F720E0A2E7B0E001C01D92AF39B20756
:1000B000E1F7A2D2BDC2A4CFCF93DF9360918500B8
:1000C000635067FDA2C080918200CCE0D0E0C81BE5
:1000D000D109C757DF4F809181008D3209F084C06C
:1000E000683009F090C083EC809375008AE58093B6
:1000F0006100109272008881807619F0CE0129D2B9
:1001000060C08A8110927E009981911106C0109280
:100110007F002EE730E082E050C0953019F48093E4
:1001200086003DC09630A9F59B81913019F488E393
:1001300090E004C0923041F486E290E09093840015
:100140008093830082E121C09330F1F4811108C0D3
:1001500080E890E0909384008093830084E015C051
:10016000813041F480E690E0909384008093830096
:1001700080E20BC0823041F48AE490E090938400E6
:100180008093830086E101C080E090E49093720048
:1001900018C0983079F0993031F4809388002EE7B8
:1001A00030E080E00AC081E09A3009F080E02EE77C
:1001B00030E003C028E830E081E0309384002093F1
:1001C00083008F3F39F4988197FD8E8190E890935A
:1001D000720007C09F81911104C09E81981708F496
:1001E000892F809360000FC08091720087FF0BC041
:1001F000CE01E5D18F3F21F48EE18093610003C0F1
:10020000811110926000109285008091610084FF3E
:1002100046C0809160008F3F09F441C0C82F8930EB
:1002200008F0C8E08C1B809360008091750098E80E
:10023000892780937500CC2331F120918300309180
:1002400084008091720086FF0BC0A6E7B0E0F90140
:100250008C2F8A0F94919D9331968A13FBCF09C0FE
:10026000D901E6E7F0E08C2F8E0F9D9191938E13CC
:10027000FCCF8FEF8C0F90E00196820F931F90932D
:100280008400809383006C2F86E790E031D0CC5FB0
:10029000CC3019F08FEF80936000C093610084E14F
:1002A00090B39C7031F48150D9F71092860010926F
:1002B0008000DF91CF91089585B7826085BF8BB7AD
:1002C00080648BBF0895A82FB92F80E090E041E0B3
:1002D00050EA609530E009C02D9182279795879567
:1002E00010F084279527305EC8F36F5FA8F3089558
:1002F000EADF8D939D930895CF93CFB7CF93C395A6
:10030000839BE9F7839B09C0839B07C0839B05C040
:10031000839B03C0839B01C0A1C0DF93C091820077
:10032000DD27C757DF4F839B02C0DF91EBCF2F93B1
:100330000F931F9300B32FEF03FB20F94F933F93CD
:1003400010B34FEF012703FB21F93BE031C04E7F93
:10035000012F10B3216028C0102F4D7F22600000B4
:1003600000B329C04B7F2460012F000010B32BC0C5
:1003700010B3477F28602AC04F7E00B320612CC095
:100380004F7D10B320622FC04F7B00B3206432C07A
:10039000422700B349934FEF0000102713FB20F9C9
:1003A00010B31C70C9F1297F91F2012703FB21F9D9
:1003B00000B3237F89F2315058F1102713FB22F943
:1003C00010B3277E79F2012703FB23F92F7C81F2FA
:1003D00000B3102713FB24F92F7971F200C010B37A
:1003E000012703FB25F92F7359F200C000B3102732
:1003F00013FB26F9223040F200C010B3012703FBA3
:1004000027F9243028F64F77206810B30000F9CF81
:1004100010E41ABF002717C03B503195C31BD040D2
:1004200010E41ABF0881033CE9F00B34D9F02091A5
:1004300080001981110F1213EDCF093641F10D32F1
:1004400011F0013E39F7009387003F914F911F91C2
:100450000F912F91DF91CAB7C6FD51CFCF91CFBF7A
:10046000CF91189520918700222379F31091850070
:10047000112311F5343012F130938500209381005F
:10048000109182003BE0311B3093820017C0009135
:10049000850001308CF40AE53091610034FD10C014
:1004A00000936100C5E7D0E00FC02795A8F4515034
:1004B000A9F4220F0000F9CF4AE503C042ED01C0C4
:1004C000432FC4E1D0E032E011B31C60939A11BB1A
:1004D00002B320E41CE05F93012756E002BB27959E
:1004E00020F4515021F4220FF9CF012756E00000EB
:1004F0003B5A02BBD0F2279528F4515029F4220F21
:100500000000F9CF012756E0279502BB20F4515097
:1005100021F4220FF9CF012756E02991332302BBA2
:1005200021F6037F10918600110FC651D04002BB07
:1005300011F01093800010E41ABF086011B3137F0C
:10054000402F437F5F9100C000C002BB11BB42BB84
:100550007CCFFC018181823071F030F4882349F036
:10056000813049F5C09A27C0833069F08430C1F0EA
:1005700022C0C098089582E690E090938400809312
:10058000830080E108958281809369008381809354
:100590006A00848180936B00858180936C000BC01E
:1005A00086818093730010927400813130F080E175
:1005B0008093730002C080E008958FEF089520912A
:1005C0007300382FFC01A0917400A21738F0A0939B
:1005D000740081E0A21779F080E0089591E09A0F0D
:1005E0008E2F831B861798F78191B0E0AE59BF4FCD
:1005F0008C93A92FEACF089581E087BB2EE088E194
:1006000090E00FB6F894A89581BD0FBE21BD54DED1
:100610008B9A8AEFA895EFE6F7E13197F1F700C0E2
:1006200000008150B9F78B987894A89545DDFDCFEF
:04063000F894FFCF6C
:10063400FF5A48656C6C6F2C205553422100000012
:020644000000B4
:00000001FF
